:030000000219FDE5
:03000B000200AA46
:03002B000201656A
:03005B000202F8A6
:030073000202DEA8
:1000800002030406080C10182030406080040608A3
:100090000C10182030406080A0C000070F1F3F0DDB
:1000A0000D04050D050305030302C2AFC0D0C0E077
:1000B000206217E5256002E473E525F4F58A758B67
:1000C00000D262D0E0D0D0D2AF3285268AC262E5BB
:1000D00026F46035306803207210758B00D0E0D0B4
:1000E000D0D295D293D297D2AF32D295D293D29723
:1000F000206E0C2066097406D5E0FDE57E42907501
:100100008B00D0E0D0D0D2AF32758A00C28DD262DF
:1001100001FF01B9306805206602C29501B9306857
:1001200005206602C29701B9306805206602C293B5
:1001300001B9C29430680A2066077406D5E0FDC292
:100140009501B9C29630680A2066077406D5E0FDAD
:10015000C29701B9C29230680A2066077406D5E0DA
:10016000FDC29301B9C2AFC2AD53E6EFC0D0C0E04B
:10017000D2D3D2AFC2CEE52A6007207449152A2116
:10018000C67800790020742EE580307E01F430E5D9
:100190000278FF53DACF207E0343DA20307E034318
:1001A000DA10C2D8C271E580307E01F430E5027900
:1001B000FFC3E89970CB306103752A18207403756A
:1001C0002A18885FD27020740DE52B6004152B214E
:1001D000D643DA01C2D82070024134A85F20610200
:1001E000C2702074367982B70431C3E894F04003BA
:1001F00074F0F8E8C4540F28F87984B70302411B5F
:10020000C313C3138721200802C313200A06C3C8DF
:1002100098F8411B28F8500374FFF88822E52D5404
:10022000066011E533C313C31324062522F52250BB
:10023000037522FF7882B60459852224A824C3E5D9
:100240002495644002A864C3E895664002A86688C5
:1002500025E56970024185C3E8AA699A5003E8FA66
:10026000E4F9EAC333FBE56BF45B29400D256AF83A
:10027000E56A6002156A400B41850AC3E56A9A5037
:1002800002056A78FF8826C26EC3E52694F840020C
:10029000D26EC3E52594404002D26420CF0AD0E05C
:1002A000D0D043E610D2AD32C2CF053A7801E52A6C
:1002B0006005307402152AC3E55F9401400575623C
:1002C0000041D4756300756C00E5622401F562504D
:1002D000037562FFD0E0D0D043E610D2AD32C2AF9A
:1002E000C0D053E67FC260759100855694855795BE
:1002F000759104D0D0D2AF32C2AF53E6EFC2ADC0D9
:10030000D0C0E0C0F0D2D3D2AFA8FBA9FCC2D83095
:100310007102615F53DACF207E0343DA10307E032F
:1003200043DA20D271E580307E01F420E5026136A7
:1003300088278928A18653DACF207E0343DA20302C
:100340007E0343DA10C2D8C271307402A172780001
:10035000E580307E01F430E502A172885FA15A5336
:10036000DACF207E0343DA20307E0343DA10C271F5
:10037000206102813853DACF207E0343DA10307EC9
:100380000343DA20C2D8D271885A895BC3E89558F2
:10039000F8E99559F97B007E087A00C3E8948CE966
:1003A00094005005755E00812A882178A2E6A82174
:1003B0006055C3E894C8E994005008E4D2E4FB7A9D
:1003C0000A8105C3E89468E994015008E4D2E3FB8C
:1003D0007A0F8105C3E894D0E994025008E4D2E290
:1003E000FB7A1E8105C3E894A0E994055008E4D285
:1003F000E1FB7A3C8105C3E89498E994085008E44D
:10040000D2E0FB7A787E00C3E8955CFCE9955DFD5F
:1004100030E70AECF42401FCEDF43400FD755E00D5
:10042000C3EC9AED9E5003755E01885C895D855A28
:1004300058855B597802A15AC3E89527F8E99528B1
:10044000F9307C02A13E307B02A13E307A02A13716
:10045000207502815BE9FDE8FC817AE9C313F9E8C4
:1004600013F8307902A137E9C313F9E813F83078AB
:0F04700002A137E9C313FDE813FC206126C3EC9A
:10047F00941CED940240028191ED7018C3EC94C866
:10048F0050120529C3E529940A5002A172755F0025
:10049F00D270A172E529600215297888E6F97400F7
:1004AF00207F087896B90302789EE624FAFEE4349A
:1004BF0000FFC3EC9EFCED9FFD9208B90310A2084C
:1004CF005007207609D27681DD307602C276A208F7
:1004DF005016B9030DECF42401FCEDF43400FD02C9
:1004EF0004F778007900A13EB90315EC33FCED3326
:1004FF00FDC3EC940AFCED9400FD50047C007D00DC
:10050F00C3EC94FFED9400400678FF7900A13EEC18
:10051F008575F0A4C5F0A2F733F879004003020502
:10052F005A78FF790002055AE9C313F9E813F83036
:10053F007C0EE9600278FFC3E81338F8E43400F961
:10054F00C3E894FFE99400400278FF885FD27020DF
:10055F006102A172741FF4552F4BF52FC274EB700B
:10056F0002D274752A18307403752A0A306102A1F9
:10057F008620740353DAFE207403752B06D0F0D057
:10058F00E0D0D0D2AD43E6103279010205B679033F
:10059F000205B6790A0205B6791E0205B67964021C
:1005AF0005B679C80205B67817E4D5E0FDD8FAD9B3
:1005BF00F6227A147B780205DD7A107B8C0205DD3A
:1005CF007A0D7BB40205DD7A0B7BC80205DD79025B
:1005DF00B27DE4C296D5E0FDC297D5E0FDD297D5A6
:1005EF00E0FDD296D5E0FDC295E576D5E0FDD2953A
:1005FF007496D5E0FDD9D9EAF8D5E0FDD8FBDBCE6E
:10060F00C29622C37C007D0075F00005F0EA33FA34
:10061F00EB33FB50F6EB13FBEA13FAC3E9FFE8FEEB
:10062F00E89AF8E99BF95004EFF9EEF8B3EC33FCD4
:10063F00ED33FDD5F0DFEDF9ECF822E889F08A20F3
:10064F00D2D4F8A9F07B0030F70B7BFFF42401F82C
:10065F00E9F43400F9E88520F0A4ADF0F8E985203D
:10066F00F0A4AFF0FEED2EF974003FFA7C04C3EA5C
:10067F0013FAE913F9E813F8DCF48BF030F70AE812
:10068F00F42401F8E9F43400F9E889F0C2D4F8A9A8
:10069F00F0227882B604030206FCC3E55F940140A2
:1006AF00030206C6852224E4F545F546F547F548CD
:1006BF00F549C26D0206FC7882E6FCD26DE522F5A3
:1006CF0023783879C7AA40AB41C3EB13FBEA13FA7F
:1006DF00EC146013C3EB13FBEA13FAEC141460076A
:1006EF00C3EB13FBEA13FAD1128845894622C3E5FF
:1006FF00459523F8E5469400F9500CC3E89480E93A
:10070F0094FF401602072DC3E8947FE9940050032D
:10071F0002072D787F790002072D788079FF884AAC
:10072F00894B22E54A2547F8E54B3548F9854B209B
:10073F00E4300701F43549FA30E709C3EA94F04091
:10074F001502076BC3EA940F500302076B78FF790A
:10075F00FF7A0F02076B780079007AF0C3E52495D2
:10076F0064500AC374019524500B020789E54B208E
:10077F00E70E020789E54B30E706884789488A4923
:10078F002278A4E6FAC3E54A33F8E54B33F9D14AA8
:10079F00E930E70BC3E89480E994FF4013E1C3C34A
:1007AF00E8947FE994005002E1C3787F7900E1C3B8
:1007BF00788079FFE820E715C3E52398F84009C34F
:1007CF00E8940140030207EA78010207EAE8F424FB
:1007DF00012523F840030207EA78FF884C2278A509
:1007EF00E6FAA848A949D14AE930E70CC3E89401D1
:1007FF00E994FF401602081EC3E894FFE9940050E5
:10080F000302081E78FF790002081E780179FFE9BC
:10081F0020E715C3E54C98F84009C3E8940140035D
:10082F000208457801020845E8F42401254CF840F8
:10083F000302084578FF88242278FFC26420693DAF
:10084F00206A12D264C3E541940A4009C3E5259496
:10085F00405002C26479A1E76023E541601F74FF35
:0F086F008541F0848539F0306A0375F005A4F8EF
:10087E00C5F0600278FFC3E895675002A8678866E6
:10088E0022C3E5409440E5419401E566500314010E
:10089E00A0046002F566220208A82275E89022786C
:1008AE0083E6FFE5E820ECF7A8BDA9BE0573C3E516
:1008BE007394084052757300E9FA79A0E76044EA30
:1008CE007007E574601B0208E3C3E895746010E5D9
:1008DE00745006600C140208EF0460F90208EFE58C
:1008EE0074F574C3946D401B7564C0C394044013B7
:1008FE00756480C39404400B756440C39404400334
:10090E0075640075BB0822E5642410500274FFF56F
:10091E00647982B70402213CC3A864E5249850028E
:10092E00A824C3E895664002A86688258826E57344
:10093E00B4070375BB1022743279A687F0A4C5F0F4
:10094E00A2F733F8C3E895644002A864882288248D
:10095E00882588268867227540007541F022C2AF2F
:10096E0075C820A8CCA9CDAA3A30CF010A75C824E3
:10097E00D2AFAB3BAC3C883B893CC3E89BF8E99CCF
:10098E00206908F9306702418121DEAD3D8A3DF9CB
:10099E00EA9DFA600478FF79FFAE3EAF3F8B3E8C46
:1009AE003FC3EC9FFCC3E99CF542A83BA93CC3E8BE
:1009BE009EF8E99FF9C3E54113FBE54013FAE82AD7
:1009CE00F540E93BF54150067540FF7541FF412862
:1009DE00AA40AB41AC40AD417E047F02C3EB940410
:1009EE0040021E1FC3EB940840021E1FC3ED13FDF1
:1009FE00EC13FCDEF7C3EA9CFAEB9DFBEF6009C338
:100A0E00E913F9E813F8DFF7EA28FAEB39FB8A4025
:100A1E008B4150067BFF8B408B41C3EB94025002FF
:100A2E00D2673069047F0341537892E6FFC3E537FE
:100A3E00948240110FC3E53794A040010FC3EF9489
:100A4E000640027F057E05E541C4540FF9E541C419
:100A5E0054F0F8E540C4540F28F8C3E89EFAE99420
:100A6E0000FB4009C3EA9402EB940050047A02E4BE
:100A7E00FB41CDAA40AB41EBC4FEEAC4540F4EFC81
:100A8E00C3EA9CFAEB9400FBC3E813C313F8EA28FD
:100A9E00FAEB3400FB8A408B41C3EB94024002C256
:100AAE00677805EBC4FE7B00EAC4540F4EFAC3EA26
:100ABE0098FA4005C3940250027A027892E6FF300B
:100ACE00600241CD855256855357D26043E680C3AE
:100ADE00E49AF8E49BF93067026167E8FAE9FBD320
:100AEE00E913FDE813FC88528953C3EF9403603871
:100AFE00EF20E00DE82CF8E93DF9ECFAEDFB020BE6
:100B0E0022E828F8E939F9C3E82402F8E93400F9B3
:100B1E007AFE7BFFC3EF9403400E8A548B55884EAA
:100B2E00894F8C508D51619B885489558A4E8B4FBD
:100B3E008C508D51306920C3E53394034019E54242
:100B4E00A2E713F8E555F4240138400B20E70875A9
:100B5E0054FFF42401F555619BE8FAD3E813FC88A1
:100B6E0052C3EF94036020EF20E007E82CF8ECFA74
:100B7E006187E8282402F87AFEC3EF940340088ABE
:100B8E0054884E8C50619B88548A4E8C50E56BC3B2
:100B9E00335002646BF56B30600261A5753402D27E
:100BAE006043E680E52D54066026A840A941C3E9BE
:100BBE0013F9E813F8C2AF53E67F759100C3E498BA
:100BCE00F594E499F595759104D26043E680D2AF21
:100BDE0022D265754400752000306B0375204002EB
:100BEE000BFED265754400752040306B03752000F6
:100BFE00D2AF7801206722E52D54066002C265C38C
:100C0E00E541940540137802940540087803940555
:100C1E0040027806306902780A206019E5446015B2
:100C2E0030690AC3E53394034003D53406D2AFD2FC
:100C3E006C81CF71ADD2AF0000C2AF206726E54107
:100C4E00C3FB940F40027B0FEB240530730123305E
:100C5E006A02742820620123F93069027982E58BD9
:0F0C6E00C39940B50544E59B5440B5200281B9B8
:100C7D0030690A08C3E8940A4001088127206502FB
:100C8D0061FEC26553E67F75910030671075940063
:100C9D007595FE759104D26043E68061FEAE40AF5E
:100CAD0041C3E49EF594E49FF59581A0C3E533948B
:100CBD0002500261FE30650261FED80281CD8127AE
:100CCD00C26C53E67F759100855494855595759149
:100CDD0004854E56854F57D26043E680D2AFE52D41
:100CED0054066008206A020533020D09306C0D2090
:100CFD006B0A206507158115810215742278003065
:100D0D0064053065027801E53775F007A4F9E5F063
:100D1D0028F5F0E9A2F013A2F113A2F213F537C3EF
:100D2D0094785003753778C3E53795384008D26607
:100D3D00D295D293D297306002A1438550568551FA
:100D4D0057D26043E68022207D11C2AF754302C2A7
:100D5D0096D294D2AF759F11020F23C2AF75430285
:100D6D00C296D292D2AF759F11020F2330724320DB
:100D7D007D20C2AF754303900143757E40D293C26F
:100D8D0092306204C297A197D296D2AF759F13028B
:100D9D000F23C2AF754303900143757E40D295C2B8
:100DAD0094306204C297A1B7D296D2AF759F10024C
:100DBD000F23207D17C2AF75430390011ED29330D0
:100DCD006202C297D2AF759F13020F23C2AF754354
:100DDD000390011ED295306202C297D2AF759F105B
:100DED00020F23207D11C2AF754304C294D292D25B
:100DFD00AF759F10020F23C2AF754304C292D294F8
:100E0D00D2AF759F13020F23307243207D20C2AFE6
:100E1D00754305900132757E10D297C296306204EB
:100E2D00C295C133D294D2AF759F11020F23C2AFB9
:100E3D00754305900154757E04D297C296306204B5
:100E4D00C293C153D292D2AF759F11020F23207D51
:100E5D0017C2AF754305900114D297306202C29547
:100E6D00D2AF759F11020F23C2AF754305900128B4
:100E7D00D2973062EBC293D2AF759F11020F232030
:100E8D007D11C2AF754306C292D296D2AF759F1334
:100E9D00020F23C2AF754306C294D296D2AF759F8F
:100EAD0010020F23307242207D20C2AF7543019096
:100EBD000154757E04D295C294306204C293C1CFA1
:100ECD00D292D2AF759F10020F23C2AF754301901E
:100EDD000132757E10D293C292306204C295C1EF79
:100EED00D294D2AF759F13E123207D16C2AF754307
:100EFD0001900128D295306202C293D2AF759F1036
:100F0D00E123C2AF754301900114D293306202C246
:100F1D0095D2AF759F13C26622900112757E00D2D5
:100F2D0095D293D297C294C292C296C26222788011
:100F3D0076090876090876040876FF0876030876A0
:100F4D00FF08760A087603087601087601788C7614
:100F5D00010876FF0876FF0876FF0876FF0876FF12
:100F6D000876030876FF0876FF0876FF08762508D1
:100F7D0076D00876280876500876040876FF08762D
:100F8D000208760008767A0876FF08760108760161
:100F9D00087600087603227887E6FFC272BF030247
:100FAD00D2727888E6C394036008C27DE630E10210
:100FBD00D27DC27E7889E630E102D27EC3EF940203
:100FCD006008758E01D273020FDC758E00C273221C
:100FDD007880E6149000809378A4F67881E61490DA
:100FED0000809378A5F67886E61490008D9378A608
:100FFD00F6789CE67538FF75390CB402067538A085
:10100D0075390AB4030675388275390578A3E61467
:10101D0090009A93F569120F2622227896E6FA78B7
:10102D0097E6FB7888E6B40305C3EB940EFB307F9F
:10103D00047A007BFFC3EB9AFCC3948250027C823E
:10104D007575000575EC8575F0A4C3E5F0947D40CC
:10105D00F222D27F11281205A77A007B007C101294
:0F106D00059DE55F2AFA74003BFBDCF37C04C3AE
:10107C00EB13FBEA13FADCF7FEC27F112822E5EF33
:10108C0020E6037520000520903FFFE52014600644
:10109C00901DFF1460009304600375EF1253D9BFC9
:1010AC007581C043FF8012059875EF0243B203E5CA
:1010BC00B3240420E70DF521E5E320E0068521B3F8
:1010CC0043E301120F267580FF75A40075F1B2750C
:1010DC00D4DF7590A975A5FC75F2FE75D50175A6C2
:1010EC000175E241E4F8F6D8FD756B01120F3B1265
:1010FC0015B678988676753001C2AF1205B1120517
:10110C00C11205A71205C81205A71205CF1205A713
:10111C00C2AF78FA79FA308507D9FBD8F7021C00F0
:10112C00120FA4120FDD1127112878988676120F52
:10113C002675885075891275C82475910475D84028
:10114C0075A82275B80275E690759B80759D007523
:10115C00D10E75BC5875BB0875BA1175E8801205AF
:10116C0098D2AF1208A553DACF207E0343DA203091
:10117C007E0343DA1043DA01C2D8C2711205B1D230
:10118C00617B037A0CE55E70077A0CDB0302111CA1
:10119C001205A720700302111CC270E55FC39402F4
:1011AC0040E1E52F541F856160F561B560D5DAD556
:1011BC00C26153DACF207E0343DA20307E0343DA58
:1011CC0010C2D8C27178A2E67008D274E52F54E030
:1011DC00F52FC2757529001205AC307409C3E529C9
:1011EC00940A4002D27512059D7802307402780080
:1011FC00C3E55F9840F0C2AF1205C11205C11205DC
:10120C00C1D2AF1205B1754D007888E6B403024126
:10121C00F312059D788CE6C3940150030212F3E59A
:10122C0030C3940150030212F3207435C3E55F946C
:10123C00FF50030212F3C2AF1205D6D2AF1205ACA7
:10124C00C3E55F940150EFC2AF1205C11205A212A3
:10125C0005C1D2AF1205ACC3E55F94FF40E902179C
:10126C005E7F02D27F11281205ACC2AFC27F11285B
:10127C00AE5FC3E55F947FD2AF4076120598C2AFE4
:10128C001205D6D2AFDFDC115FC3EE94057897F66A
:10129C001205B11215F81216E17F0AD27F1128122D
:1012AC0005ACC2AFC27F1128AE5FC3E55F947FD29D
:1012BC00AF50E6120598C2AF1205C11205A2120575
:1012CC00C1D2AFDFD6115FEE24057896F61205B1C8
:1012DC001215F81217101205AC1128C3E55F94FF14
:1012EC005002413502175EC3E55F954D4003855FA3
:1012FC004D1205AC78017988E7B403027805C3E593
:10130C005F9840024115C2AF1205D61205D61205E0
:10131C00D6D2AF1205B1753000E4F531F532053196
:10132C00E531F470390532789AE678191460127840
:10133C003214600D787D14600878FA1460037532ED
:10134C0000C3E53298401715327531B4789986761A
:10135C00C2AF1205D6D2AF789886761205AC1205BC
:10136C00A2E52A7005307402211C780120740278E1
:10137C0006C3E55F9840A77888E6C3940360031220
:10138C0005ACE52A700302111CC2AF120F26E4F55E
:10139C0022F523F524F525F526F56AD2AF7885E6F6
:1013AC00C333F568E4F545F546F547F548F549F5D9
:1013BC0073F52CF52DF53775730875BB1012059860
:1013CC001208A9E5E820ECFBA8BDA9BEE97001F85C
:1013DC0088741208AD75730875BB107887E6FE76B5
:1013EC0002120FA47887EEF6C2AF7564FF1209459E
:1013FC00852264852265852266D2AF75220175240B
:10140C000175250175260185636C756D017888E67B
:10141C00B40307C27D307602D27DD268D2697533AF
:10142C0000120E8C120EB112096512096C120965AC
:10143C0012096C120965021452C2AF120FA4D2AF7A
:10144C0075730075BB08120BF01206A1120D0A126F
:10145C000D5412096C120BDF306D031206FD206760
:0D146C000312084830670312088F120D0AA2
:10147900120D7912096C120BF0306D03120732123A
:101489000D0A120DF012096C120BDF306D031207F1
:1014990090120D0A120E1512096C120BF0306D0321
:1014A9001207ED120D0A120E8C12096C1208A912FC
:1014B9000BDF120D0A120EB11208AD12096C306958
:1014C90035206B3285676485676585636C756D0149
:1014D90079187A0CC3E53399400FC269D26A8A3503
:1014E9008567648567660214FFC3E55F940140035D
:1014F90002145202157C306A1B206B18E5351470F2
:1015090004C26A8145F535C3E55F940140030214BD
:101519005202157C753600C3E56278FA985054304A
:101529007404E52A604D7888E6B40317207D052008
:101539007607A14C307602A14C206B07D26B8567E8
:1015490064819178F0306B058567647820C3E54143
:101559009850028152306B1BC26BC27D307602D229
:101569007DD26A75351285676481520536E55F60FB
:1015790002A17F753600C2AF120F267887E6FE7684
:1015890002120FA47887EEF6E4F522F523F524F587
:1015990025F526F568C268D2AF120598120F2630D4
:1015A9007409C3E53694054002211C6125901A0D82
:1015B900782012163AE520B4550CA312163AE52004
:1015C900B4AA030215D8120F3B1215F80215F790A9
:1015D9001A0378807B0A12163AA308DBF9901A0FCE
:1015E900788C7B1812163AA308DBF9901A2722C2C5
:1015F900AF121679121653901A00740E12163FA3E1
:10160900740412163FA3741412163F901A037880BB
:101619007B0A12163EA308DBF9901A0F788C7B1807
:1016290012163EA308DBF912168C12166A901A27B5
:1016390022E493F622E6438F01538FFD75EF02757D
:10164900B7A575B7F1F0538FFE22438F02438F017F
:1016590075EF0275B7A575B7F1901A0DF0538FFCA8
:1016690022901A0D7455D13F901A0E74AAD13F22B7
:101679007A3079D07820901A40D13AE520F709A339
:10168900DAF7227A3079D0901A40E7D13F09A3DA04
:10169900F922AB77A878BB01027980BB0202798174
:1016A900BB03027982BB04027984BB05027986BB3C
:1016B90006027992BB07027987BB080279A3BB09A5
:1016C90002799CBB0A027988BB0B027989E8F72267
:1016D9007C051205B1DCFB22C2AF1205C11205C897
:1016E9001205CF1205D61205A21205C11205C8129C
:1016F90005CF1205D61205A21205C11205C8120599
:10170900CF1205D6D2AF22C2AF1205D61205CF121B
:1017190005C81205C11205A21205D61205CF120578
:10172900C81205C11205A21205D61205CF1205C8A5
:101739001205C1D2AF22AE77AF78C2AF1205C1127E
:1017490005C11205C11205A2DEF21205D61205A2C3
:10175900DFF8D2AF22D1E1D1D9D1D9757701757826
:1017690001757900F13F7C05AD5F1205B1C3ED95B7
:101779005F70F5C3E55F9401400AC3E55F94FF40DC
:101789003202179AD19BB1F8D1E1C2AF75EF12D1EC
:10179900D9DCD50579C3E5799403500280C6D1D93E
:1017A9000578E5771490009F93F808C3E578985079
:1017B9000280AED1D9D1D90577C3E577940C50020F
:0E17C900809C120F3BB1F8C2AF75EF12D1D960
:0319FD0002108A4B
:101A00000E0414090904FF03FF0A03010155AA018A
:101A1000FFFFFFFFFF03FFFFFF25D0285004FF0259
:081A2000007AFF01010003FF41
:101A4000235475726E6967794E6665743235412329
:101A500023424C48454C4923463333302320202031
:101A60002020202020202020202020202020202076
:101C0000C2AFC2D353D9BF7581C043B20343FF8073
:101C1000752438752503B1C975EF0275E24043F1AB
:101C20002053A4DF75D400D2857DFA780379E67C51
:101C300010752200752300901DD67B0675249875BB
:101C400025013085028142208508D8FBD9F9DCF7CF
:101C500081B4308508D8FBD9F9DCF781B4B189E4C7
:101C600093A3C39A6004DDC381B4DBDBB17B600264
:101C7000812B7B08E493FAA3B15CDBF87A30B15C8A
:101C8000752200752300B17BEAFCEBFDC3ED94FEE9
:101C9000400EB17B8A278B28ED30E0048A828B834B
:101CA000B17B7AC270D8C3ED94FE601350CEBD00F4
:101CB00025EC60097520007521FF0200008100A855
:101CC00027A9280809D804D90281D3B17FEA89AAB3
:101CD000F281C50D81A0C3ED94035049EDA2E092BD
:101CE000007AC5C3E5829400E583941C50902000DF
:101CF00010438F02438F0175B7A575B7F1F030001F
:101D00001FA827A9280809438F01538FFDD804D99C
:101D100002A12089AAE275B7A575B7F1F0A3A10DBC
:101D2000538FFC817C7AC1BD030CE493A3FAB140CC
:101D3000DCF8B138817C817EAA22AB23B15CEBFA5E
:101D4000EA6222752608C3E52313F523E52213F57D
:101D50002250066323A0632201D526EAB1C9B1C986
:101D600075260AEAF4200102D285300102C285B14B
:101D7000C9C3134002C201D526EB22B17FEAFB2082
:101D80008502A17F308502A184752608AE24AF2587
:101D9000C3EF13FFEE13FEB1CDB1C9C3EA13308513
:101DA000024480FA30E703632201C3E52313F523DD
:101DB000E52213F52250066323A0632201D526D91C
:101DC000E52265236523F52222AE24AF250E0FDE22
:101DD000FEDFFCD20122424C48656C693437316326
:041DE000F3300601D5
:00000001FF
